:020000040800F2
:100000000000022009140008A1110008A91100082D
:10001000B1110008B9110008C1110008000000006A
:10002000000000000000000000000000C9110008EE
:10003000D711000800000000E5110008F3110008C6
:1000400059140008591400085914000859140008DC
:1000500059140008591400085914000859140008CC
:1000600059140008591400085914000859140008BC
:1000700059140008591400085914000859140008AC
:10008000591400085914000859140008591400089C
:1000900001120008591400085914000859140008E6
:1000A000591400085914000859140008591400087C
:1000B00015120008591400085914000859140008B2
:1000C000591400085914000859140008591400085C
:1000D000591400085914000859140008591400084C
:1000E000591400085914000859140008591400083C
:1000F000591400085914000859140008591400082C
:10010000591400085914000859140008591400081B
:10011000591400085914000859140008591400080B
:1001200059140008591400085914000859140008FB
:1001300059140008000000000000000059140008D5
:1001400059140008591400085914000859140008DB
:1001500059140008591400085914000859140008CB
:1001600059140008591400085914000859140008BB
:100170005914000859140008000000000000000095
:0801800059140008591400088D
:040188000001000171
:10018C0010B5054C237833B9044B13B10448AFF3C5
:10019C0000800123237010BD14000020000000001B
:1001AC00A859000808B5034B1BB103490348AFF32A
:1001BC00008008BD0000000018000020A8590008AD
:1001CC0053B94AB9002908BF00281CBF4FF0FF31B2
:1001DC004FF0FF3000F088B9ADF1080C6DE904CE9A
:1001EC0000F006F8DDF804E0DDE9022304B0704706
:1001FC002DE9F047089D8E4604468846002B4AD1CF
:10020C008A42174662D9B2FA82F64EB1C6F1200381
:10021C0001FA06F820FA03F3B74043EA0808B440A1
:10022C004FEA174E1FFA87FCB8FBFEF1230C0EFBAE
:10023C00118843EA084301FB0CF29A4209D9FB18D6
:10024C0001F1FF3080F0EA809A4240F2E7800239F7
:10025C003B449A1AA3B2B2FBFEF00EFB102243EA07
:10026C00024300FB0CFC9C4509D9FB1800F1FF3242
:10027C0080F0D6809C4540F2D3803B44023840EA63
:10028C000140A3EB0C0300211DB1F3400022C5E992
:10029C000032BDE8F0878B4205D90DB1C5E90001EC
:1002AC0000210846F5E7B3FA83F1002946D17345DE
:1002BC0002D3824200F20581841A6EEB0302012004
:1002CC009046002DE5D0C5E90048E2E7002A00F091
:1002DC009080B2FA82F6002E40F0A4808A1A030CA9
:1002EC004FEA174E80B2BCB20121B2FBFEFC0EFBF2
:1002FC001C2243EA024304FB0CF29A4207D9FB1876
:10030C000CF1FF3802D29A4200F2E080C4469B1AEC
:10031C00B3FBFEF20EFB123340EA034302FB04F480
:10032C009C4207D9FB1802F1FF3002D29C4200F22A
:10033C00CA8002461B1B42EA0C40A5E7C1F120060D
:10034C008B4022FA06F71F430EFA01F420FA06F34B
:10035C002EFA06FE4FEA1749234300FA01F81FFA5A
:10036C0087FCBEFBF9F01C0C09FB10EE44EA0E44B2
:10037C0000FB0CFEA64502FA01F209D93C1900F16A
:10038C00FF3A80F09C80A64540F2998002383C44AC
:10039C00A4EB0E041FFA83FEB4FBF9F309FB134420
:1003AC004EEA044403FB0CFCA44508D93C1903F1A8
:1003BC00FF3E80F08280A4457FD9023B3C4443EA57
:1003CC000040A4EB0C04A0FB02EC64457346E14630
:1003DC0062D35FD05DB1B8EB030264EB090404FA9D
:1003EC0006F622FA01F31E43CC40C5E90064002155
:1003FC004FE7B1FBF2FC010C41EA0E4180B240EA3E
:10040C0001423B4638463C46B846BE462026B1FB28
:10041C00F7F1A2EB080241EA0C4166E7014618E746
:10042C0010462CE7C6F120022EFA02F3B740B14079
:10043C0020FA02F24FEA174E0A43B3FBFEF8BCB2A5
:10044C000EFB1833110C41EA034108FB04F9B040D0
:10045C0089454FEA104380B23ED9791808F1FF3C28
:10046C0001D289451FD8A1EB0901B1FBFEF909FBAB
:10047C0004F80EFB191192B242EA0142424529D20C
:10048C00BA1809F1FF31C4D24245C2D2A9F1020116
:10049C003A44BEE7F0459DD2BEEB02036CEB070C71
:1004AC000138E14696E7A7EB09094944A8F1020C8B
:1004BC00B1FBFEF909FB04F8DBE773467FE7504616
:1004CC0066E70846FDE63B44023A33E7ACF1020C22
:1004DC003B441CE749469CE7A1EB0901C446B1FB30
:1004EC00FEF909FB04F8C4E7704700BF80B500AF04
:1004FC00174B184A1A60164B06225A60144B0022EE
:10050C009A60134B0022DA60114B4FF420221A61CF
:10051C000F4B4FF480125A610D4B00221A760C4B84
:10052C0001225A760A4B01229A76094B0122DA767D
:10053C00074B00221A77064B00225A77044802F028
:10054C0009FE0346002B01D000F0F6FD00BF80BD74
:10055C00640000200064004080B58AB000AF786071
:10056C0007F1140300221A605A609A60DA601A616B
:10057C007B681B681D4A934234D100233B611C4BA2
:10058C001B6C1B4A43F000731364194B1B6C03F078
:10059C0000733B613B690023FB60154B1B6B144ADA
:1005AC0043F002031363124B1B6B03F00203FB605B
:1005BC00FB684FF440737B610223BB610023FB613A
:1005CC0003233B6209237B6207F114031946094894
:1005DC0003F03EFE00220021142003F0F4FD142051
:1005EC0003F00DFE00BF2837BD4680BD00640040FF
:1005FC00003802400004024080B582B000AF786041
:10060C007B681B680A4A93420DD10A4B1B6C094A42
:10061C0023F0007313644FF44071074803F0B4FFE8
:10062C00142003F0FAFD00BF0837BD4680BD00BFA3
:10063C0000640040003802400004024080B400AF67
:10064C00034B1B889BB21846BD465DF8047B704774
:10065C008801000880B400AF074B1B68B3F1FF3F63
:10066C0002D1064B1B6801E0034B1B681846BD46C4
:10067C005DF8047B704700BF8CC100088C01060834
:10068C0080B58AB000AF00237B610023BB610123DE
:10069C00FB6100233B6000237B600023BB600023D5
:1006AC00FB6000233B6101233B620E237B623B46D4
:1006BC001946094802F06CFE0346002B01D000F0ED
:1006CC003BFD054802F042FF0221034803F026FAE5
:1006DC0000BF2837BD4680BD6400002080B586B0C1
:1006EC0000AFB9607A603B600346FB7302F026FDF5
:1006FC00786101233B611A4A7B681360184A7B6856
:10070C005360174B04229A60154B0022DA603B6A47
:10071C00082B01D908233B62114A3B6A136107F18C
:10072C0010033A680E490F4802F09DFF0BE002F0EF
:10073C0005FD02467B69D31A642B04D93B69194623
:10074C00084803F060F83B691946064803F0A0F826
:10075C000346002BEBD100BF00BF1837BD4680BD50
:10076C00300000206400002080B58AB002AF7860B1
:10077C007B681B68334A93425FD107F11003324AFE
:10078C000021324803F0A8F82F4B5B6840F201724D
:10079C0093420DD12C4B9B68042B09D12A4B5968E1
:1007AC00294B1B69DBB207F11002002000F0BEFEE2
:1007BC00254B5B6840F21D2293423ED1224B9B6835
:1007CC00042B3AD1FFF73AFF0346BB83204B1B782F
:1007DC00012B03D11F4B1B68FB8302E01E4B1B68D4
:1007EC00FB83FFF737FFB861BB8B1B0A9BB2DBB2F5
:1007FC003B72BB8BDBB27B72FB8B1B0A9BB2DBB2FB
:10080C00BB72FB8BDBB2FB72BB691B0EDBB23B73A7
:10081C00BB691B0CDBB27B73BB691B0ADBB2BB7302
:10082C00BB69DBB2FB7307F108030822009240F2AC
:10083C001D2202210120FFF751FF00BF2037BD46CA
:10084C0080BD00BF00640040480000206400002010
:10085C00B81E00208801060888C1000880B400AFCB
:10086C00034BF322DA6000BFBD465DF8047B704792
:10087C00003C024080B485B000AF78600023FB6080
:10088C007B68404A934206D27B68B3F1006F02D377
:10089C000023FB606FE07B683B4A934206D27B6887
:1008AC00384A934202D30123FB6064E07B68374AE9
:1008BC00934206D27B68344A934202D30223FB60F4
:1008CC0059E07B68324A934206D87B682F4A9342A0
:1008DC0002D30323FB604EE07B682E4A934206D87A
:1008EC007B682B4A934202D90423FB6043E07B686C
:1008FC00294A934206D87B68264A934202D905239B
:10090C00FB6038E07B68254A934206D87B68224A14
:10091C00934202D90623FB602DE07B68204A934268
:10092C0006D87B681D4A934202D90723FB6022E05C
:10093C007B681C4A934206D87B68194A934202D9B9
:10094C000823FB6017E07B68174A934206D87B6844
:10095C00144A934202D90923FB600CE07B68134ACA
:10096C00934206D87B68104A934202D90A23FB6053
:10097C0001E00B23FB60FB6818461437BD465DF89D
:10098C00047B7047004000080080000800C000088D
:10099C00FFFF0008FFFF0108FFFF0308FFFF05082A
:1009AC00FFFF0708FFFF0908FFFF0B08FFFF0D08FB
:1009BC0080B400AF054B064A5A60044B054A5A6096
:1009CC0000BFBD465DF8047B704700BF003C024091
:1009DC0023016745AB89EFCD80B400AF054B1B6994
:1009EC00044A43F00043136100BFBD465DF8047B2D
:1009FC00704700BF003C024080B584B000AF786007
:100A0C000023FB6002F09AFBF8600EE07B68B3F108
:100A1C00FF3F0AD07B68002B17D002F08FFB0246F9
:100A2C00FB68D31A7A689A420FD30A4BDB6803F43B
:100A3C008033002BEAD1074BDB6803F00103002B5A
:100A4C0004D0044B0122DA6000E000BF1037BD4631
:100A5C0080BD00BF003C024080B584B000AF786020
:100A6C000023FB600223FB72FB7A002B02D10023D4
:100A7C00FB6010E0FB7A012B03D14FF48073FB6019
:100A8C0009E0FB7A022B03D14FF40073FB6002E008
:100A9C004FF44073FB607B680B2B02D97B680433EB
:100AAC007B60174B1B69164A23F440731361144B7C
:100ABC001A691349FB6813430B61114B1B69104AEC
:100ACC0023F0780313610E4B1A697B68DB00134328
:100ADC000B4A43F002031361094B1B69084A43F4A8
:100AEC00803313614FF4FA60FFF786FF044B1B69E8
:100AFC00034A23F07A03136100BF1037BD4680BD53
:100B0C00003C024080B582B000AF78603960114B78
:100B1C001B69104A23F4407313610E4B1B690D4A79
:100B2C0043F4007313610B4B1B690A4A43F0010336
:100B3C0013617B683A681A600A20FFF75DFF054B6A
:100B4C001B69044A23F00103136100BF0837BD463B
:100B5C0080BD00BF003C024080B582B000AF786021
:100B6C000B46FB700F4B1B690E4A23F44073136149
:100B7C000C4B0C4A1B6913610A4B1B69094A43F065
:100B8C00010313617B68FA781A700A20FFF734FFAF
:100B9C00044B1B69034A23F00103136100BF0837A0
:100BAC00BD4680BD003C024080B582B000AF78608D
:100BBC00FFF7FEFEFFF752FE7868FFF75BFE034679
:100BCC001846FFF749FFFFF707FF002318460837C1
:100BDC00BD4680BD80B582B000AF0346FB71FB798A
:100BEC00012B10D10021012000F030F81048FFF744
:100BFC00DBFF1048FFF7D8FF0F48FFF7D5FF0F4872
:100C0C00FFF7D2FF0FE0FB79022B0CD10021022061
:100C1C0000F01CF80A48FFF7C7FF0A48FFF7C4FFAB
:100C2C000948FFF7C1FF002318460837BD4680BDB1
:100C3C0000C00008000001080000020800000408C1
:100C4C00000006080000080800000A0880B584B0FF
:100C5C0000AF03460A46FB711346BB71FB79012BAF
:100C6C0010D1BB793B73134B1B78DBB27B731248EF
:100C7C00FFF79AFF07F10C01002302220E4800F047
:100C8C001DF812E0FB79022B0FD10B4B1B78DBB25A
:100C9C003B73BB797B730848FFF786FF07F10C01A8
:100CAC0000230222044800F009F800BF1037BD46AB
:100CBC0080BD00BF018000080080000880B586B0B0
:100CCC0000AFF860B9607A60FB70FB6803F0030357
:100CDC007B61FA687B69D31AFB60FB78002B08D028
:100CEC00F868FFF761FF0346002B02D04FF0FF338B
:100CFC004DE0FFF75DFEFFF7B1FD11E0FA687B698F
:100D0C001A44BB681B7819461046FFF725FFBB68D1
:100D1C000133BB607B6901337B617B68013B7B608A
:100D2C007B6903F00303002B15D07B68002BE5D106
:100D3C0011E0FA687B691A44BB681B6819461046B7
:100D4C00FFF7E0FEBB680433BB607B6904337B6157
:100D5C007B68043B7B607B68032BEAD811E0FA6864
:100D6C007B691A44BB681B7819461046FFF7F4FEE2
:100D7C00BB680133BB607B6901337B617B68013BE2
:100D8C007B607B68002BEAD1FFF726FE0023184618
:100D9C001837BD4680BD80B582B000AF0120FFF78B
:100DAC0019FF00237B6014E07B6803F1006303F5FB
:100DBC00C0231B78DBB23B707B6803F1006000F54D
:100DCC004040394600230122FFF778FF7B6801334E
:100DDC007B607B68B3F5A82FE6D300BF00BF083754
:100DEC00BD4680BD80B584B000AF786072B600BFE0
:100DFC000023FB6010E0154AFB6860334FF0FF31B5
:100E0C0042F82310114AFB6820334FF0FF3142F8AF
:100E1C002310FB680133FB60FB68072BEBDD0C4BED
:100E2C0000221A600B4802F090FA02F00DF97B6870
:100E3C001B68BB60BB6883F3088800BF7B68043306
:100E4C001B68984700BF1037BD4680BD00E100E02D
:100E5C0010E000E06400002080B58AB000AF07F11C
:100E6C00140300221A605A609A60DA601A61002337
:100E7C003B61394B1B6B384A43F080031363364B91
:100E8C001B6B03F080033B613B690023FB60324B1F
:100E9C001B6B314A43F0010313632F4B1B6B03F0A5
:100EAC000103FB60FB680023BB602B4B1B6B2A4AC6
:100EBC0043F002031363284B1B6B03F00203BB606C
:100ECC00BB6800237B60244B1B6B234A43F0040359
:100EDC001363214B1B6B03F004037B607B681023B3
:100EEC007B610123BB610023FB6100233B6207F1A3
:100EFC0014031946194803F0ABF908237B6101234D
:100F0C00BB610023FB6100233B6207F1140319460C
:100F1C00134803F09DF904237B610023BB6100237C
:100F2C00FB6100233B6207F1140319460D4803F0E3
:100F3C008FF908237B610023BB610023FB61002335
:100F4C003B6207F114031946064803F081F900BF10
:100F5C002837BD4680BD00BF003802400008024063
:100F6C00000402400000024080B485B000AF03468C
:100F7C00FB71114B1B68FB60104B1B68BB60FB6863
:100F8C00B3F1FF3F01D10023FB60BB68B3F1FF3F1E
:100F9C0001D10023BB60FB79012B01D1FB6805E07B
:100FAC00FB79022B01D1BB6800E0002318461437F3
:100FBC00BD465DF8047B704788C1000888010608AF
:100FCC0080B582B000AF02F01DF800F04BF8FFF7CF
:100FDC0043FFFFF78BFA00F033F91C4804F084F858
:100FEC00FFF74EFB00F032FB01F0AAF90120FFF7EE
:100FFC00BBFF78600220FFF7B7FF3860144B1B78FB
:10100C00DBB2012B09D17A683B689A4205D2FFF713
:10101C00C2FE01210120FFF719FE01F043FA0D4B2E
:10102C001B6840F2DC529342F7D10B4B1B78DBB2BE
:10103C00012B07D1074B40F2DC521A600748FFF72F
:10104C00D1FEEAE7064B01221A70E6E78C0000207D
:10105C0001800008E00000200080000800C00008AB
:10106C00E400002080B594B000AF07F120033022DB
:10107C000021184604F058FC07F10C0300221A60FA
:10108C005A609A60DA601A610023BB60284B1B6CB3
:10109C00274A43F080531364254B1B6C03F0805399
:1010AC00BB60BB6800237B60224B1B68214A43F466
:1010BC00804313601F4B1B6803F480437B607B6889
:1010CC0001233B624FF480337B620223BB634FF4FA
:1010DC008003FB6304233B64A8237B640223BB646F
:1010EC000423FB6407F12003184603F049FB034675
:1010FC00002B01D000F020F80F23FB6002233B6192
:10110C0000237B614FF4A053BB614FF48053FB6110
:10111C0007F10C030521184603F0AAFD0346002B2A
:10112C0001D000F009F800BF5037BD4680BD00BFAC
:10113C00003802400070004080B400AF72B600BFAF
:10114C0000BFFDE780B483B000AF00237B60104B81
:10115C005B6C0F4A43F4804353640D4B5B6C03F49C
:10116C0080437B607B6800233B60094B1B6C084A07
:10117C0043F080531364064B1B6C03F080533B60AD
:10118C003B6800BF0C37BD465DF8047B704700BF61
:10119C000038024080B400AF00BFFDE780B400AF60
:1011AC0000BFFDE780B400AF00BFFDE780B400AF27
:1011BC0000BFFDE780B400AF00BFFDE780B400AF17
:1011CC0000BFBD465DF8047B704780B400AF00BF24
:1011DC00BD465DF8047B704780B400AF00BFBD46D0
:1011EC005DF8047B704780B500AF01F093FF00BF42
:1011FC0080BD000080B500AF024802F0B5FC00BF16
:10120C0080BD00BF6400002080B500AF024803F031
:10121C00DBFF00BF80BD00BF8C00002080B400AF9E
:10122C00064BD3F88830054A43F47003C2F8883073
:10123C0000BFBD465DF8047B704700BF00ED00E0C9
:10124C0080B586B000AF07F1080300221A605A601F
:10125C009A60DA603B4600221A605A601D4B4FF0D0
:10126C0080421A601B4B53225A601A4B00229A6020
:10127C00184B4FF47A72DA60164B00221A61154B38
:10128C0000229A61134803F0DFFE0346002B01D0C5
:10129C00FFF752FF4FF48053BB6007F10803194668
:1012AC000C4804F081F80346002B01D0FFF744FFF3
:1012BC0000233B6000237B603B461946054804F045
:1012CC00A3FA0346002B01D0FFF736FF00BF1837F7
:1012DC00BD4680BD8C00002080B584B000AF786026
:1012EC007B681B68B3F1804F15D10023FB600C4B5E
:1012FC001B6C0B4A43F001031364094B1B6C03F08A
:10130C000103FB60FB68002200211C2002F05BFF44
:10131C001C2002F074FF00BF1037BD4680BD00BF1B
:10132C000038024080B586B002AF78607B681B68DD
:10133C00B3F1804F51D100F0FBFF2A4B1B78002BEF
:10134C000FD1294B1B680133274A1360264B1B68AE
:10135C0040F2DB52934207D9234B40F2DC521A6025
:10136C0002E0214B00221A60204B1B78012B34D158
:10137C001F4B1B6801331E4A13601D4B1B68B3F5D2
:10138C007A7F2AD31A4B00221A601A4B1B68FB81F6
:10139C00194B04221A70184B50225A70164B022209
:1013AC009A70FB891B0A9BB2DAB2134BDA70FB8979
:1013BC00DAB2114B1A71104B55225A710E4B552241
:1013CC009A710D4B5522DA71082300930A4B40F2A7
:1013DC00097202210120FFF781F900BF1037BD46C9
:1013EC0080BD00BFDC000020E0000020E4000020F5
:1013FC00E800002088010008D4000020DFF834D079
:10140C00FFF70CFF0C480D490D4A002302E0D4589D
:10141C00C4500433C4188C42F9D30A4A0A4C002332
:10142C0001E013600432A242FBD304F085FAFFF70B
:10143C00C7FD7047000002200000002014000020AF
:10144C00005E000814000020C01E0020FEE7000013
:10145C0080B487B000AFF860B9607A6000237B611C
:10146C0011E0BA687B6913441B781A46FB68534039
:10147C00DBB20A4A52F82320FB681B0A5340FB607C
:10148C007B6901337B617A697B689A42E9D3FB689B
:10149C0018461C37BD465DF8047B7047D0590008D0
:1014AC0090B484B000AF03463960FB710123FB7329
:1014BC00FB791B4AD35CDBB2002B2AD0FB79184A90
:1014CC00D25CD2B2013AD1B2154AD154FA79FB7935
:1014DC001449CB5C1C463868134913469B001344D3
:1014EC005B0023441B010B4404460FCB84E80F0024
:1014FC00FB790C4AD25C0132D1B20A4AD154094A66
:10150C00D35C092B03D9FB79064A0021D154002363
:10151C00FB73FB7B18461037BD4690BC704700BF71
:10152C003002002034020020EC00002080B48BB08C
:10153C0000AFB9607A601A460346FB731346BB735F
:10154C00FB7B2F4AD35CDBB2092B26D8FB7B2C4AC6
:10155C00D25CD2B20132D1B2294AD154FA7BFB7B94
:10156C002849CB5CDBB2194613469B0013445B0045
:10157C000B441B01244A13447B62FB7B214AD25C43
:10158C00D2B20132D2B21F491046C854092A07D927
:10159C00FB7B1C4A0021D15402E007F114037B624F
:1015AC007B6ABA681A607B6ABA7B1A737B6A1B7B8C
:1015BC00002B1FD07B681A787B6A1A717B685A786B
:1015CC007B6A5A717B689A787B6A9A717B68DA7845
:1015DC007B6ADA717B681A797B6A1A727B685A7932
:1015EC007B6A5A727B689A797B6A9A727B68DA7921
:1015FC007B6ADA7200BF2C37BD465DF8047B7047FE
:10160C00300200202C020020EC00002080B483B0BB
:10161C0000AF786039607B681A783B681B789A4217
:10162C000BD17B685A783B685B789A4205D17B6812
:10163C00DA783B68DB789A4201D0002300E0012382
:10164C0018460C37BD465DF8047B704780B483B0F8
:10165C0000AF0023FB710CE0FB79194A40F618012E
:10166C0001FB03F31344143300221A70FB7901338A
:10167C00FB71FB79002BEFD00023FB7116E0FB799B
:10168C00104A40F2244101FB03F3134418330022A7
:10169C001A70FB790B4A40F2244101FB03F313440B
:1016AC001C3300221A60FB790133FB71FB79002B90
:1016BC00E5D000BF00BF0C37BD465DF8047B70471A
:1016CC0038020020500A002080B485B000AF78604A
:1016DC000023FB7318E0FB7B104A40F6180101FB5A
:1016EC0003F3134414331B78002B0AD1FB7B40F615
:1016FC00180202FB03F3094A1A447B681A600023A0
:10170C0006E0FB7B0133FB73FB7B002BE3D0012357
:10171C0018461437BD465DF8047B7047380200202C
:10172C0080B485B000AF78600023FB7318E0FB7BBE
:10173C00104A40F2244101FB03F3134418331B7885
:10174C00002B0AD1FB7B40F2244202FB03F3094A33
:10175C001A447B681A60002306E0FB7B0133FB73A1
:10176C00FB7B002BE3D0012318461437BD465DF8F4
:10177C00047B7047500A002080B584B000AF7860BD
:10178C000023FB731BE0FB7B40F6180202FB03F308
:10179C000E4A1344043379681846FFF737FF0346A3
:1017AC00002B09D0FB7B094A40F6180101FB03F31F
:1017BC001344143300221A70FB7B0133FB73FB7B45
:1017CC00002BE0D000BF1037BD4680BD3802002092
:1017DC0080B485B000AF786039600023FB7318E0EB
:1017EC00FB7B114A40F2244101FB03F313441833F1
:1017FC001B78002B0AD0FB7B40F2244202FB03F344
:10180C00094A1A443B681A60002306E0FB7B01334B
:10181C00FB73FB7B002BE3D0012318461437BD462A
:10182C005DF8047B704700BF500A002080B485B07F
:10183C0000AF786039600023FB7318E0FB7B114A22
:10184C0040F6180101FB03F3134414331B78002BEF
:10185C000AD0FB7B40F6180202FB03F3094A1A4438
:10186C003B681A60002306E0FB7B0133FB73FB7BB8
:10187C00002BE3D0012318461437BD465DF8047BDA
:10188C00704700BF3802002090B58BB002AF786073
:10189C000023FB77194B1B68FB600023FB7715E0DB
:1018AC00FB7F9AB27B681B899A4205D27B685A6887
:1018BC00FB7F13441B7801E0114B1B78FA7F20321D
:1018CC003A4402F8103CFB7F0133FB77FB7F072B7C
:1018DC00E6D908233B760B4B18780B4B1968FA6842
:1018EC003B7E1C4607F10C0304330094FEF7F6FE16
:1018FC00002318462437BD4690BD00BFE85D0008A4
:10190C00EC5D0008DC5D0008E05D000890B58BB074
:10191C0000AF78607B6807F114040FCB84E80F00EC
:10192C00002387F827307B681A8997F82730591CD1
:10193C0087F82710D2B228333B4403F81C2C002321
:10194C0087F8263013E07B685A6897F826301A44DB
:10195C0097F82730591C87F82710127828333B4406
:10196C0003F81C2C97F82630013387F8263097F8AB
:10197C0026309AB27B681B899A42E4D307F10C0398
:10198C00BB6197F827309BB2BB8307F11403184651
:10199C00FFF77AFF034618462C37BD4690BD000072
:1019AC0090B58BB000AF7860002387F827307B6848
:1019BC0007F1080408330FCB84E80F0007F1180374
:1019CC00FB607B6822333B627B681B8A1B0A9BB2E1
:1019DC00DAB2F96897F82730581C87F827000B44BF
:1019EC0042F01002D2B21A707B68198AFA6897F822
:1019FC002730581C87F827001344CAB21A700BE022
:101A0C003B6A5A1C3A62F96897F82720501C87F8F1
:101A1C0027000A441B78137097F82730072BEFD94F
:101A2C0008233B8207F108031846FFF72DFF0346F6
:101A3C00002B0AD17B6804221A76064B1A887B6825
:101A4C001A847B683A6ADA6000BF00BF2C37BD4647
:101A5C0090BD00BFD45D000890B58DB000AF78602C
:101A6C00002387F82F307B6807F10C0408330FCB69
:101A7C0084E80F0007F11C033B617B68DB68BB62E9
:101A8C007B689B88002B06D07B689B88013B9AB2B5
:101A9C007B689A8082E07B685A887B689A807B6836
:101AAC009B795A1CD1B27A6891715BB203F00F0327
:101ABC005BB243F0200359B23A6997F82F30581CA7
:101ACC0087F82F001344CAB21A707B681A8A7B6895
:101ADC00D9687B682233CB1A9BB2D31AFB84FA8C5D
:101AEC0097F82F30C3F108039A4202DAFB8CDBB271
:101AFC0004E097F82F30C3F10803DBB287F82530E8
:101B0C0097F8252097F82F30134487F825300BE0F1
:101B1C00BB6A5A1CBA62396997F82F20501C87F897
:101B2C002F000A441B78137097F82F2097F8253054
:101B3C009A42EDD397F825309BB2BB8207F10C0388
:101B4C001846FFF7A1FE0346002B0FD1154B1A8840
:101B5C007B681A847B68BA6ADA607B685B78013BC5
:101B6C00DAB27B685A707B681B78002B7B681A8A08
:101B7C007B68D9687B682233CB1A9BB2D31AFB845F
:101B8C00FB8C002B09D17B68DB6900221A707B6807
:101B9C00054ADA617B6800221A7600BF3437BD46ED
:101BAC0090BD00BFD65D0008740E002090B585B0C6
:101BBC0000AF786039603B6802221A7007F10803A5
:101BCC001846FFF7ADFD0346002B36D13B680122CA
:101BDC001A700023FB810DE07B685A68FB89D118D1
:101BEC00BA68FB89097813440A4683F82220FB89DA
:101BFC000133FB817B681B89FA899A42ECD3BB6861
:101C0C007A6803F1080413460FCB84E80F00BA6816
:101C1C00BB682232DA60BB6801221A76BB680122EB
:101C2C009A71BB683A68DA61BB68064A12881A84F2
:101C3C00BB681846FFF7B4FE00E000BF1437BD4682
:101C4C0090BD00BFD05D000880B58AB000AF786051
:101C5C007B689B89B3F5006F06D9022387F8273080
:101C6C007B6807221A7505E0002387F827307B680C
:101C7C0006221A7507F10C03BB61BB6997F8272084
:101C8C0042F03002D2B21A70BB690133174A127893
:101C9C001A70BB690233164A12781A700323BB837D
:101CAC00144B1B783B757B681B797B757B68DB79E8
:101CBC00FB757B689B79BB7507F114031846FFF71E
:101CCC00E3FD0346002B0CD10B4B1A887B68DA82A0
:101CDC007B681B7D062B01D1052200E000227B686E
:101CEC001A7500BF2837BD4680BD00BFED5D0008EA
:101CFC00EE5D000808000020D85D000880B582B0B9
:101D0C0000AF78607B685B681B78002B15D07B6814
:101D1C001B897A685268127893420ED97B685B688B
:101D2C001B781A467B681A817B685B685A1C7B6837
:101D3C005A60786800F010FB00E000BF0837BD4621
:101D4C0080BD000090B585B000AF78607868FFF773
:101D5C0013FD07F108031846FFF7B6FC0346002BEA
:101D6C004ED17B685B681B781BB21B021BB203F461
:101D7C0070631AB27B685B6801331B781BB2134328
:101D8C001BB2BB81BB89072B3CD97B685B689A1C57
:101D9C007B685A607B681B89023B9AB27B681A810C
:101DAC00BB6800221A70BB687A681C1D13460FCBE7
:101DBC0084E80F00BB68BA899A81BA68BB6818328C
:101DCC009A600023FB730CE07B685A68FB7BD1188C
:101DDC00BA689368581C90600A781A70FB7B0133C0
:101DEC00FB73FB7B9AB27B681B899A42ECD3BB6872
:101DFC00064A1288DA82BB681846FFF725FF02E014
:101E0C0000BF00E000BF1437BD4690BDD25D000896
:101E1C0080B586B000AF786007F10C03194678687E
:101E2C00FFF704FD0346002B68D1FB681B7D052BD7
:101E3C0066D1FB681A780132D2B21A701A787B68B4
:101E4C005B681B785340DBB203F00F03002B51D1BE
:101E5C007B685B685A1C7B685A607B681B89013BFA
:101E6C009AB27B681A81FB681833FA6892891A4413
:101E7C00FB689B68D31ABB827B681B89BA8A9A421F
:101E8C0003D97B681B89DBB201E0BB8ADBB2FB7434
:101E9C000023FB750CE07B685A68FB7DD118FA684F
:101EAC009368581C90600A781A70FB7D0133FB759F
:101EBC00FA7DFB7C9A42EED3FB681833FA68928960
:101ECC001A44FB689B68D31ABB82BB8A002B0CD1CB
:101EDC00FA68FB6818329A60FB680433184600F005
:101EEC003BFAFB6800221A750BE0FB68064A128865
:101EFC00DA8206E0FB6800221A7502E000BF00E0FF
:101F0C0000BF1837BD4680BDD85D000880B584B0D1
:101F1C0000AF786007F10C0319467868FFF758FC9E
:101F2C000346002B73D1FB681B7E042B71D17B689D
:101F3C001B89022B6FD97B685B681B7803F00F033E
:101F4C00002B02D0012B48D056E0FB6803221A76F6
:101F5C007B685A68FB6852781A70FA68FB681278CA
:101F6C005A707B685B6802331B785BB2002B06DB14
:101F7C007B685B6802331A78FB685A8012E07B68D6
:101F8C005B6802331B78F02B09D97B685B680233E2
:101F9C001B78F92B03D8FB6801225A8002E0FB68FE
:101FAC007F225A80FA68FB6852885A80FB685B88EB
:101FBC001A461C4B1B88DBB292FBF3F2FB6892B205
:101FCC005A80FA68FB6852889A80FB68164A128815
:101FDC001A84FB680022DA7120E0FB6804221A766E
:101FEC00FB68124A12881A84FB68DA790132D2B281
:101FFC00DA71DB79042B10D9FB6800221A76FB68A6
:10200C00DB6902221A70FB68094ADA6106E000BF3C
:10201C0004E000BF02E000BF00E000BF1037BD4687
:10202C0080BD00BFDA5D0008D65D0008D45D0008F5
:10203C00740E002080B588B000AF78607B681B6898
:10204C00002B22DB7B6804333B617B681B7BBB82F0
:10205C000023BB737B681B6840F2DF72934204D190
:10206C007723FB73F1233B730FE07B681A68244BD7
:10207C001B689A4209D17623FB73F1233B737B686F
:10208C001B68DBB22133DBB27B733B691B781B090A
:10209C00FB77FB7B772B02D0FB7BDB2B02D1FB7F0F
:1020AC00002B29D1FB7F032B27D8FB7F032B24D8B4
:1020BC0001A252F823F000BFD5200008E12000084F
:1020CC00ED200008F920000807F10C031846FFF773
:1020DC0015FE12E007F10C031846FFF733FE0CE077
:1020EC0007F10C031846FFF793FE06E007F10C030B
:1020FC001846FFF70BFF00E000BF2037BD4680BD40
:10210C00E45D000880B582B000AF786039603B6850
:10211C00002B01D1134B3B60134B1A787B681A7060
:10212C007B681B89072B0BD87868FFF7EFFB0346FE
:10213C00002B01D1002200E002223B681A700CE057
:10214C007B681B89B3F5806F04D839687868FFF712
:10215C002DFD02E03B6802221A7000BF0837BD4615
:10216C0080BD00BF740E00200800002080B582B036
:10217C0000AF0023FB7165E0FB79364A40F2244145
:10218C0001FB03F3134418331B78012B02D0032BF0
:10219C000BD015E0FB7940F2244202FB03F32D4AED
:1021AC0013441846FFF7FCFB0AE0FB7940F224428B
:1021BC0002FB03F3274A13441846FFF74DFC00BFFC
:1021CC00FB79244A40F2244101FB03F313442033EE
:1021DC001B88002B14D0FB791E4940F2244203FBD0
:1021EC0002F20A4420321288013A90B2194A40F2A3
:1021FC00244101FB03F31344203302461A801EE0F2
:10220C00FB79144A40F2244101FB03F313441833C5
:10221C0000221A70FB790F4A40F2244101FB03F3B0
:10222C0013441C331B6802221A70FB79094A40F2D2
:10223C00244101FB03F313441C33074A1A60FB7956
:10224C000133FB71FB79002B96D000BF00BF083720
:10225C00BD4680BD500A0020740E002080B586B0AB
:10226C0000AF03E03B1D1846FFF7E4FE3B1D19468B
:10227C000020FFF715F90346002BF3D00023FB7564
:10228C004CE0FB7D294A40F6180101FB03F3134493
:10229C0014331B78062B0AD0FB7D244A40F6180118
:1022AC0001FB03F3134414331B78072B09D1FB7D7B
:1022BC0040F6180202FB03F31C4A13441846FFF7BE
:1022CC00C3FCFB7D194A40F6180101FB03F31344D0
:1022DC0016331B88002B14D0FB7D144940F61802D2
:1022EC0003FB02F20A4416321288013A90B20F4AEA
:1022FC0040F6180101FB03F31344163302461A800F
:10230C0009E0FB7D094A40F6180101FB03F3134475
:10231C00143300221A70FB7D0133FB75FB7D002BFF
:10232C00AFD000BF00BF1837BD4680BD38020020BB
:10233C0080B500AFFFF792FFFFF718FF00BF80BD1D
:10234C0080B400AF034B02221A7000BFBD465DF88B
:10235C00047B70470900002080B582B000AF786024
:10236C007B681A89474B1A817B68DB68454AD360C6
:10237C007B6859687B681B891A46434803F000FB4D
:10238C00404B414A5A607B685B681B78113B262B9B
:10239C0068D801A252F823F04124000871240008E7
:1023AC0071240008712400087124000871240008AD
:1023BC00712400087124000871240008712400089D
:1023CC00712400087124000871240008712400088D
:1023DC00712400087124000871240008712400087D
:1023EC00712400087124000871240008712400086D
:1023FC00712400087124000871240008712400085D
:10240C007124000871240008712400084924000874
:10241C00712400087124000851240008712400085C
:10242C007124000859240008712400086124000854
:10243C0069240008154B01221A701FE0144B01226D
:10244C001A701BE0134B01221A7017E0124B012279
:10245C001A7013E0114B01221A700FE0104B01227D
:10246C001A700BE07B68DB78762B07D17B685B6896
:10247C001B781121184600F057F800BF00BF083731
:10248C00BD4680BD780E0020880E0020881E0020DE
:10249C00891E00208A1E00208B1E00208C1E00200E
:1024AC008D1E002080B500AF194B1B78012B05D178
:1024BC00174B00221A70174800F05AF8164B1B786D
:1024CC00012B05D1144B00221A70124800F0DEF8D3
:1024DC00124B1B78012B05D1104B00221A700D48A2
:1024EC0000F00AFB0E4B1B78012B05D10C4B002284
:1024FC001A70084800F0DEFB0A4B1B78012B05D143
:10250C00084B00221A70034800F036FD00BF80BD56
:10251C00881E0020780E00208A1E00208B1E0020B2
:10252C008C1E00208D1E002080B58AB000AF0346A3
:10253C000A46FB711346BB710C4B1B687B6207F19F
:10254C001003FB617F233B74FB797B74BB79BB74F9
:10255C0003233B8407F10F0207F1180311461846B9
:10256C00FFF7D0FD00BF2837BD4680BDE85D0008F1
:10257C0080B58AB000AF7860002387F8273007F168
:10258C000C03BB610623BB750C237B757B68DB7866
:10259C00772B02D17723FB7501E07623FB753A4B41
:1025AC001B78012B07D17B685B681B787F21184651
:1025BC00FFF7BAFF65E07B681B89022B07D07B68AD
:1025CC005B681B7813211846FFF7AEFF59E07B6858
:1025DC005B6801331B7823F07F0387F826307B6818
:1025EC005B6801331B7803F07F0387F8253097F87D
:1025FC002530012B02D0032B1CD037E0012387F8A8
:10260C0027307B685B681B784033DBB23B737B689D
:10261C005B685B787B730223BB8397F82630802B37
:10262C002CD007F10B0207F1140311461846FFF7E3
:10263C0069FD23E0012387F827307B685B681B78F2
:10264C004033DBB23B737B685B685B787B73022344
:10265C00BB8397F82630802B12D007F10B0207F1C1
:10266C00140311461846FFF74DFD09E07B685B68C3
:10267C001B7812211846FFF757FF02E000BF00E05D
:10268C0000BF2837BD4680BD0900002080B590B042
:10269C0000AF786007F1200300221A605A609A603C
:1026AC00DA6007F10C0300221A605A609A60DA6053
:1026BC001A610023FB72002387F83F30002387F850
:1026CC003E30062387F822300C2387F8213007F19F
:1026DC000C037B627B68DB78772B03D1772387F83D
:1026EC00233002E0762387F823307B68002B07D059
:1026FC007B685B68002B03D07B681B89032B04D899
:10270C0013213120FFF710FFF2E17B685B68013386
:10271C001B7803F07F0387F8373097F83730012B9D
:10272C0007D07B685B681B7812211846FFF7FCFE0C
:10273C00DEE17B685B6802331B781BB21B021AB2AA
:10274C007B685B6803331B781BB213431BB2BB86DD
:10275C00BB8EB3F57F4F3CD0B3F57F4F00F39D811B
:10276C0040F60F62934200F00881B3F5616F80F27E
:10277C00948140F60E62934200F0D18040F60E62D6
:10278C00934200F38A8140F20222934200F0888047
:10279C0040F20322934240F080817B681B89042B1A
:1027AC0007D07B685B681B7813211846FFF7BCFECB
:1027BC009EE1A24B01221A70002387F83E30A04BF9
:1027CC0000221A709F4B00221A70012387F83F30A9
:1027DC006BE17B681B890D2B07D07B685B681B78D2
:1027EC0013211846FFF7A0FE82E17B685B68053376
:1027FC001B781A067B685B6806331B781B041A432C
:10280C007B685B6807331B781B0213437A6852683A
:10281C000832127813431A468B4B1A607B685B683C
:10282C0009331B781A067B685B680A331B781B0418
:10283C001A437B685B680B331B781B0213437A6863
:10284C0052680C32127813431A46804B1A607E4B36
:10285C001B687F4A934204D17C4B1B68B3F5A82FAD
:10286C0007D97B685B681B7831211846FFF75CFE43
:10287C003EE10220FEF7AEF938633B6B002B14BF30
:10288C0001230023DBB287F83E3097F83E30002B53
:10289C0002D16B4B01221A70012387F83F3004E1FF
:1028AC007B681B89082B07D07B685B681B7813211E
:1028BC001846FFF739FE1BE17B685B6804331B7815
:1028CC001A067B685B6805331B781B041A437B680C
:1028DC005B6806331B781B0213437A685268073215
:1028EC00127813431A465B4B1A605A4B1A685A4BB0
:1028FC001B689A4214BF01230023DBB287F83E30D9
:10290C0097F83E30002B03D14E4B01221A7002E097
:10291C004C4B00221A70012387F83F30C5E07B68CE
:10292C001B89042B07D07B685B681B781321184626
:10293C00FFF7FAFDDCE07B685B681B784033DBB2A9
:10294C003B737B685B685B787B737B685B689B78AD
:10295C00BB737B685B68DB78FB7300233B740523DC
:10296C003B8507F10B0207F1200311461846FFF7D0
:10297C00C9FB3748FEF736FA97E07B681B89042BB6
:10298C0007D07B685B681B7813211846FFF7CCFDDA
:10299C00AEE02E4B1B68B3F5A82F7ED2FEF7FBF9E9
:1029AC002D4B4FF0FF321A600023BB6315E0BB6B5D
:1029BC0003F1006303F540431B78DBB23B72264BFB
:1029CC001B6807F1080101221846FEF741FD03467A
:1029DC00214A1360BB6B0133BB631C4B1B68BA6B86
:1029EC009A42E4D31B4B1A681B4B1B689A4235D195
:1029FC007B685B681B784033DBB23B737B685B683E
:102A0C005B787B737B685B689B78BB737B685B686C
:102A1C00DB78FB7300233B7405233B8507F10B022A
:102A2C0007F1200311461846FFF76CFB012101202A
:102A3C00FEF70CF90648FEF7D5F92EE0DC00002075
:102A4C00A81E0020B81E0020A01E0020A41E0020DE
:102A5C0000C00008B01E0020040000207B685B68EA
:102A6C001B784033DBB23B737B685B685B787B73B2
:102A7C007B685B689B78BB737B685B68DB78FB73FC
:102A8C0001233B7405233B8507F10B0207F120035F
:102A9C0011461846FFF736FB2AE07B685B681B780B
:102AAC0031211846FFF740FD22E097F83F30012B0B
:102ABC001ED17B685B681B784033DBB23B737B6851
:102ACC005B685B787B737B685B689B78BB737B68AC
:102ADC005B68DB78FB7397F83E303B7405233B85D2
:102AEC0007F10B0207F1200311461846FFF70AFB0A
:102AFC004037BD4680BD00BF80B58AB000AF78605E
:102B0C00002387F8273007F10C03BB617B681B8916
:102B1C000B2B07D07B685B681B7813211846FFF7DB
:102B2C0003FDAEE0584B1B78012B07D07B685B682C
:102B3C001B7824211846FFF7F7FCA2E07B685B6842
:102B4C005A78524B1A707B685B689A78504B1A70A3
:102B5C007B685B6803331B781A067B685B680433FD
:102B6C001B781B041A437B685B6805331B781B02BC
:102B7C0013437A685268063212781343454A13603D
:102B8C007B685B6807331B781A067B685B680833C5
:102B9C001B781B041A437B685B6809331B781B0288
:102BAC0013437A6852680A32127813433A4A136014
:102BBC00394B1B688022B3FBF2F101FB02F29B1A2A
:102BCC00002B07D1344B1B688022B3FBF2F3334A42
:102BDC00136007E0304B1B688022B3FBF2F3013328
:102BEC002E4A13602B4B1B682D4A934239D12A4B2A
:102BFC001B68B3F5A82F34D8264B2A4A1A60012338
:102C0C0087F827307B685B681B784033DBB23B73FB
:102C1C007B685B685B787B738023FF2B0AD98023EE
:102C2C001B0A9BB2DBB2BB738023DBB2FB730423A6
:102C3C00BB8304E08023DBB2BB730323BB83124B47
:102C4C0002221A70184B00221A80184B4FF0FF32D8
:102C5C001A60174B00221A6097F82730012B08D006
:102C6C000FE07B685B681B781F211846FFF75CFC44
:102C7C0007E007F10B0207F1140311461846FFF7A2
:102C8C0041FA2837BD4680BDA81E00208E1E0020AC
:102C9C008F1E0020901E0020941E0020981E0020E5
:102CAC0000C0000800000608AC1E00200400002034
:102CBC009C1E002080B5ADF5815D84B000AF07F19E
:102CCC00300343F82C0C002307F5815202F10D025E
:102CDC001370002307F5815202F10E02138007F5E1
:102CEC00805303F1100307F5805202F11C021360AC
:102CFC00994B1B78022B0AD007F1300353F82C3C6C
:102D0C005B681B7824211846FFF70EFC1FE107F1C6
:102D1C00300353F82C3C5B6801331B781A468F4BFD
:102D2C001A808E4B1B88002B0ED18D4B1B88FF2BD2
:102D3C001DD007F1300353F82C3C5B681B787321D2
:102D4C001846FFF7F1FB02E1844B1B881A46844BB3
:102D5C001B8801339A420AD007F1300353F82C3CFC
:102D6C005B681B7873211846FFF7DEFBEFE07B4BAB
:102D7C001A887B4B1A80002307F5815202F10E0250
:102D8C00138021E007F1300353F82C3C5B6807F506
:102D9C00815202F10E02128802321A4407F5815355
:102DAC0003F10E031B88127807F130010B4403F872
:102DBC00242C07F5815303F10E031B88013307F50F
:102DCC00815202F10E02138007F5815303F10E03B9
:102DDC001A8807F1300353F82C3C1B89023B9A42AA
:102DEC00D0DB604B186807F1300353F82C3C1B897F
:102DFC00023B1A4607F11003043B1946FEF728FB69
:102E0C000346584A136080231A46574B1B6803FB32
:102E1C0002F2564B1B68D01807F1300353F82C3CC8
:102E2C001B89023B1A4607F1100104390023FDF7F8
:102E3C0045FF07F5815303F10803186007F581532B
:102E4C0003F108031B68002B63D107F1300353F81F
:102E5C002C3C1B891A46464B1B681344023B444AC4
:102E6C001360012307F5815202F10D02137007F173
:102E7C00300353F82C3C5B681B784033DBB207F50E
:102E8C00805202F11002137007F1300353F82C3CFE
:102E9C005B685B7807F5805202F111021370314BBD
:102EAC001B681B0EDBB207F5805202F11202137085
:102EBC002C4B1B681B0CDBB207F5805202F1130282
:102ECC001370284B1B681B0ADBB207F5805202F10A
:102EDC0014021370234B1B68DBB207F5805202F10E
:102EEC0015021370062307F5815213801E4B1B68C5
:102EFC0001331D4A13601C4B1A681E4B1B689A4207
:102F0C0003D1154B03221A700EE0134B02221A70D8
:102F1C000AE007F1300353F82C3C5B681B787021F6
:102F2C001846FFF701FB12E007F5815303F10D037F
:102F3C001B78012B0BD107F5805202F10F0207F51C
:102F4C00805303F1180311461846FFF7DBF807F519
:102F5C0081571037BD4680BDA81E0020AA1E002038
:102F6C00AC1E0020040000209C1E0020901E00209F
:102F7C00B41E0020981E002080B58AB000AF786087
:102F8C0007F11003FB610623BB760C237B767B6871
:102F9C001B89012B07D07B685B681B7813211846B3
:102FAC00FFF7C2FA24E0144B1B78032B07D07B6885
:102FBC005B681B7824211846FFF7B6FA18E07B688B
:102FCC005B681B784033DBB23B7401233B8407F115
:102FDC000F0207F1180311461846FFF793F8064B3A
:102FEC0000221A70054B00221A60054B00221A8031
:102FFC002837BD4680BD00BFA81E00209C1E0020A7
:10300C00AC1E002080B500AF0E4B1B680D4A43F47C
:10301C00007313600B4B1B680A4A43F48063136004
:10302C00084B1B68074A43F480731360032001F0BC
:10303C00BFF80F2000F03EF8FEF784F80023184686
:10304C0080BD00BF003C024080B500AF114B124A5E
:10305C001A62104B00221A620E4B104A5A620D4B28
:10306C0000225A620B4B0E4A1A610A4B00221A615B
:10307C00084BC1225A61074B00225A61054B0122B1
:10308C009A61044B00229A6100F00CF80023184658
:10309C0080BD00BF00380240FFC9FEF633797704CB
:1030AC00FF11602080B400AF00BFBD465DF8047B0B
:1030BC007047000080B582B000AF7860124B1A6880
:1030CC00124B1B7819464FF47A73B3FBF1F3B2FB36
:1030DC00F3F3184601F0AFF80346002B01D001239F
:1030EC000EE07B680F2B0AD8002279684FF0FF3076
:1030FC0001F069F8064A7B681360002300E00123A5
:10310C0018460837BD4680BD000000201000002086
:10311C000C00002080B400AF064B1B781A46064BFF
:10312C001B681344044A136000BFBD465DF8047B62
:10313C00704700BF10000020BC1E002080B400AF00
:10314C00034B1B681846BD465DF8047B704700BFF7
:10315C00BC1E002080B584B000AF78607B68002B6B
:10316C0001D10123EDE07B6893F82030DBB2002B1A
:10317C0002D17868FDF7F0F97B681B681A687B68E8
:10318C001B6842F001021A60FFF7D8FFF86012E0EA
:10319C00FFF7D4FF0246FB68D31A0A2B0BD97B68C6
:1031AC005B6A43F400327B685A627B68052283F8C1
:1031BC0020200123C5E07B681B685B6803F00103DA
:1031CC00002BE5D07B681B681A687B681B6822F0B3
:1031DC0002021A60FFF7B2FFF86012E0FFF7AEFFD1
:1031EC000246FB68D31A0A2B0BD97B685B6A43F443
:1031FC0000327B685A627B68052283F82020012309
:10320C009FE07B681B685B6803F00203002BE5D131
:10321C007B681B7E012B08D17B681B681A687B6856
:10322C001B6842F080021A6007E07B681B681A6812
:10323C007B681B6822F080021A607B685B7E012B26
:10324C0008D17B681B681A687B681B6842F04002D7
:10325C001A6007E07B681B681A687B681B6822F0A1
:10326C0040021A607B689B7E012B08D17B681B682F
:10327C001A687B681B6842F020021A6007E07B68C2
:10328C001B681A687B681B6822F020021A607B6836
:10329C00DB7E012B08D17B681B681A687B681B6876
:1032AC0022F010021A6007E07B681B681A687B68C2
:1032BC001B6842F010021A607B681B7F012B08D13F
:1032CC007B681B681A687B681B6842F008021A60EE
:1032DC0007E07B681B681A687B681B6822F0080291
:1032EC001A607B685B7F012B08D17B681B681A68AE
:1032FC007B681B6842F004021A6007E07B681B685D
:10330C001A687B681B6822F004021A607B689A6852
:10331C007B68DB681A437B681B691A437B685B69B3
:10332C0042EA03017B685B685A1E7B681B680A4390
:10333C00DA617B6800225A627B68012283F82020C4
:10334C00002318461037BD4680BD80B582B000AF53
:10335C0078607B68002B01D1012315E0786800F0C0
:10336C0039F97868FDF748F97B681B681A687B683F
:10337C001B6842F400421A607B6800225A627B6828
:10338C00002283F82020002318460837BD4680BD54
:10339C0080B487B000AF786039607B6893F82030D8
:1033AC00FB75FB7D012B03D0FB7D022B40F0BE8017
:1033BC00654B3B613B69D3F8003243F001023B693A
:1033CC00C3F800223B69D3F8003223F47C523B69EA
:1033DC00C3F800223B69D3F800223B685B6A1B02EE
:1033EC001A433B69C3F800223B685B6903F01F0377
:1033FC00012202FA03F3FB603B69D3F81C22FB6841
:10340C00DB431A403B69C3F81C223B68DB69002B89
:10341C0023D13B69D3F80C22FB68DB431A403B6990
:10342C00C3F80C223B68DB6819043B685B689BB2F1
:10343C003A68526919433B69483243F832103B6889
:10344C009B6819043B681B689AB23B685B690A432A
:10345C0039694833DB000B445A603B68DB69012B4C
:10346C0022D13B69D3F80C22FB681A433B69C3F8A1
:10347C000C223B681B6819043B685B689BB23A687A
:10348C00526919433B69483243F832103B689B68D8
:10349C0019043B68DB689AB23B685B690A4339697B
:1034AC004833DB000B445A603B689B69002B09D105
:1034BC003B69D3F80422FB68DB431A403B69C3F831
:1034CC00042207E03B69D3F80422FB681A433B69EA
:1034DC00C3F804223B681B69002B09D13B69D3F864
:1034EC001422FB68DB431A403B69C3F8142207E043
:1034FC003B69D3F81422FB681A433B69C3F81422C6
:10350C003B681B6A012B07D13B69D3F81C22FB6873
:10351C001A433B69C3F81C223B69D3F8003223F0F1
:10352C0001023B69C3F80022002306E07B685B6A5A
:10353C0043F480227B685A62012318461C37BD462F
:10354C005DF8047B704700BF0064004080B584B018
:10355C0000AF78607B6893F82030DBB2012B2ED162
:10356C007B68022283F820207B681B681A687B68C2
:10357C001B6822F001021A60FFF7E0FDF86012E010
:10358C00FFF7DCFD0246FB68D31A0A2B0BD97B68CC
:10359C005B6A43F400327B685A627B68052283F8CD
:1035AC002020012312E07B681B685B6803F0010399
:1035BC00002BE5D17B6800225A62002306E07B6871
:1035CC005B6A43F400227B685A6201231846103769
:1035DC00BD4680BD80B584B000AF78607B6893F841
:1035EC002030DBB2022B33D17B681B681A687B68F6
:1035FC001B6842F001021A60FFF7A0FDF86012E0B0
:10360C00FFF79CFD0246FB68D31A0A2B0BD97B688B
:10361C005B6A43F400327B685A627B68052283F84C
:10362C00202001231BE07B681B685B6803F001030F
:10363C00002BE5D07B681B681A687B681B6822F03E
:10364C0002021A607B68012283F82020002306E026
:10365C007B685B6A43F480127B685A6201231846CC
:10366C001037BD4680BD80B489B000AFF860B9603A
:10367C007A603B60FB6893F82030FB77FB681B6833
:10368C009B68BB61FB7F012B03D0FB7F022B40F0BF
:10369C00AD80BB6903F08063002B0AD1BB6903F0DA
:1036AC000063002B05D1BB6903F08053002B00F0A5
:1036BC009580BB691B0E03F003037B6101227B69C0
:1036CC009A403B681A60BB689B68002B0DD1BB68A5
:1036DC001B685A05BB68DB68F96809681A437B6983
:1036EC0018331B010B441A600FE0BB685B68DA00EF
:1036FC00BB689B681A43BB68DB68F96809681A43A6
:10370C007B6918331B010B441A60FB681968BB6892
:10371C001A697B6918331B010B4404331A60BB68AC
:10372C001B7D012B11D1FB681A687B6918331B01B7
:10373C00134404331B68FA68116843F480727B6984
:10374C0018331B010B4404331A607B6807331B7856
:10375C001A067B6806331B781B041A437B680533F7
:10376C001B781B0213437A68043212781046FA68ED
:10377C00116843EA00027B691B010B4403F5C67315
:10378C001A607B6803331B781A067B6802331B783C
:10379C001B041A437B6801331B781B0213437A68A2
:1037AC0012781046FA68116843EA00027B691B0123
:1037BC000B4403F5C4731A60FB681A687B691833F1
:1037CC001B0113441B68FA68116843F001027B6902
:1037DC0018331B010B441A6000230EE0FB685B6A74
:1037EC0043F40012FB685A62012306E0FB685B6A33
:1037FC0043F48022FB685A62012318462437BD46E5
:10380C005DF8047B704780B485B000AF7860396098
:10381C007B6893F82030FB73FB7B012B02D0FB7B86
:10382C00022B28D13B6803F00103002B07D07B68E7
:10383C001B689A687B681B6842F080029A603B6840
:10384C0003F00203002B07D07B681B689A687B6827
:10385C001B6842F400429A603B6803F00403002B9F
:10386C0007D07B681B689A687B681B6842F400026F
:10387C009A60002306E07B685B6A43F480227B68D5
:10388C005A62012318461437BD465DF8047B704715
:10389C0080B485B000AF786039600023FB607B6832
:1038AC0093F82030FB72FB7A012B02D0FB7A022BAF
:1038BC000BD17B681B689A683B689B061A403B6877
:1038CC009B069A4201D00123FB60FB681846143713
:1038DC00BD465DF8047B704780B487B000AFF860DC
:1038EC00B9607A603B60FB6893F82030FB75FB7D18
:1038FC00012B03D0FB7D022B40F00381BB68002B16
:10390C000ED1FB681B68DB6803F00303002B16D198
:10391C00FB685B6A43F40012FB685A620123F7E010
:10392C00FB681B681B6903F00303002B07D1FB68C2
:10393C005B6A43F40012FB685A620123E8E0FB68FF
:10394C001A68BB681B331B0113441B6803F0040289
:10395C007B689A607B689B68002B0CD1FB681A68AB
:10396C00BB681B331B0113441B685B0DC3F30A02BA
:10397C007B681A600BE0FB681A68BB681B331B0181
:10398C0013441B68DB0823F060427B685A60FB68B9
:10399C001A68BB681B331B0113441B6803F002023B
:1039AC007B68DA60FB681A68BB681B331B01134425
:1039BC0004331B6803F00803002B03D07B68082238
:1039CC001A610BE0FB681A68BB681B331B011344BC
:1039DC0004331B6803F00F027B681A61FB681A68DA
:1039EC00BB681B331B01134404331B681B0ADAB27C
:1039FC007B689A61FB681A68BB681B331B01134414
:103A0C0004331B681B0C9AB27B685A61FB681A68FA
:103A1C00BB681B01134403F5DC731B68DAB23B680B
:103A2C001A70FB681A68BB681B01134403F5DC733E
:103A3C001B681A0A3B680133D2B21A70FB681A6809
:103A4C00BB681B01134403F5DC731B681A0C3B6841
:103A5C000233D2B21A70FB681A68BB681B0113449C
:103A6C0003F5DC731B681A0E3B680333D2B21A7071
:103A7C00FB681A68BB681B01134403F5DE731A68F4
:103A8C003B680433D2B21A70FB681A68BB681B011E
:103A9C00134403F5DE731B681A0A3B680533D2B274
:103AAC001A70FB681A68BB681B01134403F5DE73BC
:103ABC001B681A0C3B680633D2B21A70FB681A6882
:103ACC00BB681B01134403F5DE731B681A0E3B68BD
:103ADC000733D2B21A70BB68002B08D1FB681B6885
:103AEC00DA68FB681B6842F02002DA6007E0FB68CA
:103AFC001B681A69FB681B6842F020021A610023DC
:103B0C0006E0FB685B6A43F48022FB685A6201237F
:103B1C0018461C37BD465DF8047B704780B485B0F1
:103B2C0000AF786039607B6893F82030FB73FB7BC7
:103B3C00012B02D0FB7B022B09D17B681B685969D6
:103B4C007B681B683A680A435A61002306E07B686D
:103B5C005B6A43F480227B685A620123184614374F
:103B6C00BD465DF8047B704780B58AB000AF7860C5
:103B7C0000237B627B681B685B693B627B681B680C
:103B8C005B68FB617B681B689B68BB617B681B681F
:103B9C00DB687B617B681B681B693B617B681B680E
:103BAC009B69FB603B6A03F00103002B7CD0BB6973
:103BBC0003F00103002B23D07B681B6801229A6061
:103BCC00BB6903F00203002B03D0786800F083F983
:103BDC0016E0BB6903F00403002B04D07B6A43F4AA
:103BEC0000637B620CE0BB6903F00803002B04D07C
:103BFC007B6A43F480537B6202E0786800F089F9B9
:103C0C00BB6903F48073002B24D07B681B684FF4D2
:103C1C0080729A60BB6903F40073002B03D0786840
:103C2C0000F063F916E0BB6903F48063002B04D049
:103C3C007B6A43F400537B620CE0BB6903F40063C2
:103C4C00002B04D07B6A43F480437B6202E07868EB
:103C5C0000F069F9BB6903F48033002B24D07B6836
:103C6C001B684FF480329A60BB6903F40033002B5D
:103C7C0003D0786800F043F916E0BB6903F48023A5
:103C8C00002B04D07B6A43F400437B620CE0BB69DD
:103C9C0003F40023002B04D07B6A43F480337B6253
:103CAC0002E0786800F049F93B6A03F00803002B46
:103CBC000CD07B6903F01003002B07D07B6A43F414
:103CCC0000737B627B681B681022DA603B6A03F02E
:103CDC000403002B0BD07B6903F00803002B06D0E8
:103CEC007B681B680822DA60786800F030F93B6A60
:103CFC0003F00203002B09D07B681B68DB6803F020
:103D0C000303002B02D07868FCF72EFD3B6A03F00E
:103D1C004003002B0CD03B6903F01003002B07D0A1
:103D2C007B6A43F480637B627B681B6810221A6198
:103D3C003B6A03F02003002B0BD03B6903F0080314
:103D4C00002B06D07B681B6808221A61786800F08B
:103D5C0012F93B6A03F01003002B09D07B681B6837
:103D6C001B6903F00303002B02D0786800F0F9F80C
:103D7C003B6A03F40033002B0BD0FB6903F01003F8
:103D8C00002B06D07B681B6810225A60786800F004
:103D9C00FCF83B6A03F48033002B0BD0FB6903F077
:103DAC000803002B06D07B681B6808225A607868D1
:103DBC0000F0F5F83B6A03F40043002B7BD0FB6961
:103DCC0003F00403002B72D03B6A03F48073002BC6
:103DDC0008D0FB6803F00103002B03D07B6A43F08F
:103DEC0001037B623B6A03F40073002B08D0FB6871
:103DFC0003F00203002B03D07B6A43F002037B62C7
:103E0C003B6A03F48063002B08D0FB6803F00403C7
:103E1C00002B03D07B6A43F004037B623B6A03F400
:103E2C000063002B43D0FB6803F07003002B3ED0E3
:103E3C00FB6803F07003602B2BD0602B2ED8502B1B
:103E4C0022D0502B2AD8402B19D0402B26D8302BDF
:103E5C0010D0302B22D8102B02D0202B05D01DE0F7
:103E6C007B6A43F008037B6219E07B6A43F0100322
:103E7C007B6214E07B6A43F020037B620FE07B6A79
:103E8C0043F040037B620AE07B6A43F080037B6271
:103E9C0005E07B6A43F480737B6200E000BF7B68C3
:103EAC001B689A697B681B6822F070029A617B68B8
:103EBC001B6804225A607B6A002B08D07B685A6A04
:103ECC007B6A1A437B685A62786800F072F800BF0C
:103EDC002837BD4680BD80B483B000AF786000BF8A
:103EEC000C37BD465DF8047B704780B483B000AFDF
:103EFC00786000BF0C37BD465DF8047B704780B41A
:103F0C0083B000AF786000BF0C37BD465DF8047B12
:103F1C00704780B483B000AF786000BF0C37BD46EB
:103F2C005DF8047B704780B483B000AF786000BF4D
:103F3C000C37BD465DF8047B704780B483B000AF8E
:103F4C00786000BF0C37BD465DF8047B704780B4C9
:103F5C0083B000AF786000BF0C37BD465DF8047BC2
:103F6C00704780B483B000AF786000BF0C37BD469B
:103F7C005DF8047B704780B483B000AF786000BFFD
:103F8C000C37BD465DF8047B704780B483B000AF3E
:103F9C00786000BF0C37BD465DF8047B704780B479
:103FAC0083B000AF786000BF0C37BD465DF8047B72
:103FBC00704780B483B000AF786000BF0C37BD464B
:103FCC005DF8047B7047000080B485B000AF78606A
:103FDC007B6803F00703FB600C4BDB68BB60BA68C3
:103FEC004FF6FF031340BB60FB681A02BB68134318
:103FFC0043F0BF6343F40033BB60044ABB68D36037
:10400C0000BF1437BD465DF8047B704700ED00E03F
:10401C0080B400AF044BDB681B0A03F0070318469F
:10402C00BD465DF8047B704700ED00E080B483B0C2
:10403C0000AF0346FB7197F90730002B0BDBFB79C4
:10404C0003F01F02074997F907305B09012000FABA
:10405C0002F241F8232000BF0C37BD465DF8047B0B
:10406C00704700BF00E100E080B483B000AF0346AE
:10407C00FB7197F90730002B12DBFB7903F01F0261
:10408C000A4997F907305B09012000FA02F2203344
:10409C0041F82320BFF34F8F00BFBFF36F8F00BFDA
:1040AC0000BF0C37BD465DF8047B704700E100E0B3
:1040BC0080B483B000AF03463960FB7197F90730C9
:1040CC00002B0ADB3B68DAB20C4997F90730120176
:1040DC00D2B20B4483F800230AE03B68DAB20849F9
:1040EC00FB7903F00F03043B1201D2B20B441A7696
:1040FC0000BF0C37BD465DF8047B704700E100E063
:10410C0000ED00E080B489B000AFF860B9607A606F
:10411C00FB6803F00703FB61FB69C3F10703042B86
:10412C0028BF0423BB61FB690433062B02D9FB694E
:10413C00033B00E000237B614FF0FF32BB6902FAC6
:10414C0003F3DA43BB681A407B699A404FF0FF31A6
:10415C007B6901FA03F3D9437B680B401343184680
:10416C002437BD465DF8047B7047000080B582B0F3
:10417C0000AF78607B68013BB3F1807F01D30123F2
:10418C000FE00A4A7B68013B53600F214FF0FF3070
:10419C00FFF78EFF054B00229A60044B07221A6032
:1041AC00002318460837BD4680BD00BF10E000E074
:1041BC0080B582B000AF78607868FFF705FF00BF6C
:1041CC000837BD4680BD80B586B000AF0346B960E8
:1041DC007A60FB7300237B61FFF71AFF78617A68C2
:1041EC00B9687869FFF78EFF024697F90F301146D0
:1041FC001846FFF75DFF00BF1837BD4680BD80B580
:10420C0082B000AF0346FB7197F907301846FFF7F1
:10421C000DFF00BF0837BD4680BD80B582B000AF32
:10422C000346FB7197F907301846FFF71DFF00BFD7
:10423C000837BD4680BD80B582B000AF7860786825
:10424C00FFF794FF034618460837BD4680BD0000B3
:10425C0080B489B000AF7860396000237B610023A3
:10426C003B610023BB610023FB616BE10122FB6915
:10427C0002FA03F37B613B681B687A6913403B616C
:10428C003A697B699A4240F05A813B685B6803F05B
:10429C000303012B05D03B685B6803F00303022B7F
:1042AC0030D17B689B68BB61FB695B00032202FA1F
:1042BC0003F3DB43BA691340BB613B68DA68FB6903
:1042CC005B0002FA03F3BA691343BB617B68BA69FA
:1042DC009A607B685B68BB610122FB6902FA03F39D
:1042EC00DB43BA691340BB613B685B681B0903F095
:1042FC000102FB6902FA03F3BA691343BB617B68E1
:10430C00BA695A603B685B6803F00303032B17D050
:10431C007B68DB68BB61FB695B00032202FA03F379
:10432C00DB43BA691340BB613B689A68FB695B006D
:10433C0002FA03F3BA691343BB617B68BA69DA60AA
:10434C003B685B6803F00303022B23D1FB69DA089B
:10435C007B68083253F82230BB61FB6903F007031A
:10436C009B000F2202FA03F3DB43BA691340BB61D3
:10437C003B681A69FB6903F007039B0002FA03F31D
:10438C00BA691343BB61FB69DA087B680832B96907
:10439C0043F822107B681B68BB61FB695B0003223E
:1043AC0002FA03F3DB43BA691340BB613B685B68F9
:1043BC0003F00302FB695B0002FA03F3BA691343CF
:1043CC00BB617B68BA691A603B685B6803F4403375
:1043DC00002B00F0B4800023FB60604B5B6C5F4AE9
:1043EC0043F4804353645D4B5B6C03F48043FB608C
:1043FC00FB685B4AFB699B08023352F82330BB61B4
:10440C00FB6903F003039B000F2202FA03F3DB4367
:10441C00BA691340BB617B68524A93422BD07B68CC
:10442C00514A934225D07B68504A93421FD07B68F7
:10443C004F4A934219D07B684E4A934213D07B6803
:10444C004D4A93420DD07B684C4A934207D07B680F
:10445C004B4A934201D107230EE008230CE00623BC
:10446C000AE0052308E0042306E0032304E002230A
:10447C0002E0012300E00023FA6902F0030292003B
:10448C009340BA691343BB613549FB699B080233FE
:10449C00BA6941F823203B4B9B68BB613B69DB430A
:1044AC00BA691340BB613B685B6803F48013002B53
:1044BC0003D0BA693B691343BB61324ABB69936051
:1044CC00304BDB68BB613B69DB43BA691340BB61B2
:1044DC003B685B6803F40013002B03D0BA693B699B
:1044EC001343BB61274ABB69D360264B5B68BB6136
:1044FC003B69DB43BA691340BB613B685B6803F4FF
:10450C000033002B03D0BA693B691343BB611D4ACE
:10451C00BB6953601B4B1B68BB613B69DB43BA69CE
:10452C001340BB613B685B6803F48033002B03D002
:10453C00BA693B691343BB61124ABB691360FB69DF
:10454C000133FB61FB690F2B7FF690AE00BF00BF00
:10455C002437BD465DF8047B704700BF003802402D
:10456C0000380140000002400004024000080240F4
:10457C00000C0240001002400014024000180240DF
:10458C00001C0240003C014080B487B000AF786052
:10459C00396000233B610023FB600023BB600023D8
:1045AC007B61CDE001227B6902FA03F33B613A683F
:1045BC003B691340FB60FA683B699A4240F0BD804E
:1045CC00654A7B699B08023352F82330BB607B69D8
:1045DC0003F003039B000F2202FA03F3BA681340A3
:1045EC00BB607B685D4A93422BD07B685C4A9342EC
:1045FC0025D07B685B4A93421FD07B685A4A934212
:10460C0019D07B68594A934213D07B68584A93421D
:10461C000DD07B68574A934207D07B68564A934229
:10462C0001D107230EE008230CE006230AE0052342
:10463C0008E0042306E0032304E0022302E0012344
:10464C0000E000237A6902F0030292009340BA68FA
:10465C009A4232D1494B1A68FB68DB4347491340F5
:10466C000B60464B5A68FB68DB43444913404B6074
:10467C00424BDA68FB68DB4340491340CB603F4B4D
:10468C009A68FB68DB433D4913408B607B6903F000
:10469C0003039B000F2202FA03F3BB602E4A7B69D3
:1046AC009B08023352F82310BB68DA432A487B6913
:1046BC009B080A40023340F823207B681A687B6908
:1046CC005B00032101FA03F3DB431A407B681A6099
:1046DC007B69DA087B68083253F822107B6903F097
:1046EC0007039B000F2202FA03F3DB437A69D2081B
:1046FC0019407B68083243F822107B68DA687B69C2
:10470C005B00032101FA03F3DB431A407B68DA6098
:10471C007B685A6801217B6901FA03F3DB431A4079
:10472C007B685A607B689A687B695B00032101FA9D
:10473C0003F3DB431A407B689A607B6901337B612E
:10474C007B690F2B7FF62EAF00BF00BF1C37BD4619
:10475C005DF8047B704700BF003801400000024048
:10476C000004024000080240000C0240001002400D
:10477C000014024000180240001C0240003C0140A2
:10478C0080B586B000AF78607B68002B01D1012327
:10479C0067E27B681B6803F00103002B75D0884B24
:1047AC009B6803F00C03042B0CD0854B9B6803F027
:1047BC000C03082B12D1824B5B6803F48003B3F516
:1047CC00800F0BD17E4B1B6803F40033002B5BD0A6
:1047DC007B685B68002B57D1012342E27B685B68E6
:1047EC00B3F5803F06D1764B1B68754A43F4803392
:1047FC0013601DE07B685B68B3F5A02F0CD1704B88
:10480C001B686F4A43F4802313606D4B1B686C4A22
:10481C0043F4803313600BE0694B1B68684A23F444
:10482C0080331360664B1B68654A23F48023136046
:10483C007B685B68002B13D0FEF780FC386108E0C6
:10484C00FEF77CFC02463B69D31A642B01D9032387
:10485C0007E25B4B1B6803F40033002BF0D014E031
:10486C00FEF76CFC386108E0FEF768FC02463B6919
:10487C00D31A642B01D90323F3E1514B1B6803F4C6
:10488C000033002BF0D100E000BF7B681B6803F005
:10489C000203002B63D04A4B9B6803F00C03002BE4
:1048AC000BD0474B9B6803F00C03082B1CD1444BDB
:1048BC005B6803F48003002B16D1414B1B6803F09B
:1048CC000203002B05D07B68DB68012B01D0012390
:1048DC00C7E13B4B1B6823F0F8027B681B69DB00CC
:1048EC00374913430B603AE07B68DB68002B20D020
:1048FC00344B01221A60FEF721FC386108E0FEF708
:10490C001DFC02463B69D31A022B01D90323A8E1F3
:10491C002B4B1B6803F00203002BF0D0284B1B68B9
:10492C0023F0F8027B681B69DB00254913430B60FD
:10493C0015E0244B00221A60FEF700FC386108E0F9
:10494C00FEF7FCFB02463B69D31A022B01D9032369
:10495C0087E11B4B1B6803F00203002BF0D17B6833
:10496C001B6803F00803002B36D07B685B69002BB7
:10497C0016D0154B01221A60FEF7E0FB386108E0F7
:10498C00FEF7DCFB02463B69D31A022B01D9032349
:10499C0067E10B4B5B6F03F00203002BF0D01BE0C5
:1049AC00094B00221A60FEF7C9FB38610EE0FEF7D6
:1049BC00C5FB02463B69D31A022B07D9032350E1EE
:1049CC000038024000004742800E4742884B5B6F24
:1049DC0003F00203002BEAD17B681B6803F004038D
:1049EC00002B00F097800023FB75814B1B6C03F0B0
:1049FC008053002B0FD10023BB607D4B1B6C7C4A7A
:104A0C0043F0805313647A4B1B6C03F08053BB60F0
:104A1C00BB680123FB75774B1B6803F48073002B79
:104A2C0018D1744B1B68734A43F480731360FEF700
:104A3C0085FB386108E0FEF781FB02463B69D31A1F
:104A4C00022B01D903230CE16A4B1B6803F480731E
:104A5C00002BF0D07B689B68012B06D1644B1B6F3D
:104A6C00634A43F0010313671CE07B689B68052BCA
:104A7C000CD15F4B1B6F5E4A43F0040313675C4B16
:104A8C001B6F5B4A43F0010313670BE0584B1B6F22
:104A9C00574A23F001031367554B1B6F544A23F0FD
:104AAC00040313677B689B68002B15D0FEF746FB4D
:104ABC0038610AE0FEF742FB02463B69D31A41F229
:104ACC008832934201D90323CBE0494B1B6F03F08F
:104ADC000203002BEED014E0FEF730FB38610AE045
:104AEC00FEF72CFB02463B69D31A41F28832934203
:104AFC0001D90323B5E03E4B1B6F03F00203002BDF
:104B0C00EED1FB7D012B05D1394B1B6C384A23F0C0
:104B1C00805313647B689B69002B00F0A180344B9D
:104B2C009B6803F00C03082B5CD07B689B69022B01
:104B3C0041D1314B00221A60FEF700FB386108E0CE
:104B4C00FEF7FCFA02463B69D31A022B01D9032368
:104B5C0087E0274B1B6803F00073002BF0D17B68B8
:104B6C00DA697B681B6A1A437B685B6A9B011A4390
:104B7C007B689B6A5B08013B1B041A437B68DB6AFE
:104B8C001B061B4913434B601B4B01221A60FEF79B
:104B9C00D5FA386108E0FEF7D1FA02463B69D31A20
:104BAC00022B01D903235CE0114B1B6803F000734B
:104BBC00002BF0D054E0104B00221A60FEF7BEFA26
:104BCC00386108E0FEF7BAFA02463B69D31A022BA9
:104BDC0001D9032345E0064B1B6803F00073002B3F
:104BEC00F0D13DE07B689B69012B07D1012338E0B4
:104BFC000038024000700040600047421B4B5B686D
:104C0C00FB607B689B69012B28D0FB6803F4800256
:104C1C007B68DB699A4221D1FB6803F03F027B6819
:104C2C001B6A9A421AD1FA6847F6C07313407A6825
:104C3C00526A9201934211D1FB6803F440327B68B3
:104C4C009B6A5B08013B1B049A4207D1FB6803F08B
:104C5C0070627B68DB6A1B069A4201D0012300E07C
:104C6C00002318461837BD4680BD00BF00380240EF
:104C7C0080B584B000AF786039607B68002B01D1BF
:104C8C000123CCE0684B1B6803F007033A689A4297
:104C9C000CD9654B3A68D2B21A70634B1B6803F09F
:104CAC0007033A689A4201D00123B8E07B681B687D
:104CBC0003F00203002B20D07B681B6803F0040375
:104CCC00002B05D0594B9B68584A43F4E053936032
:104CDC007B681B6803F00803002B05D0534B9B68C3
:104CEC00524A43F460439360504B9B6823F0F002AC
:104CFC007B689B684D4913438B607B681B6803F092
:104D0C000103002B44D07B685B68012B07D1474B18
:104D1C001B6803F40033002B19D101237FE07B685F
:104D2C005B68022B03D07B685B68032B07D13F4B7E
:104D3C001B6803F00073002B09D101236FE03B4B80
:104D4C001B6803F00203002B01D1012367E0374BF2
:104D5C009B6823F003027B685B68344913438B60C8
:104D6C00FEF7ECF9F8600AE0FEF7E8F90246FB689A
:104D7C00D31A41F28832934201D903234FE02B4BD3
:104D8C009B6803F00C027B685B689B009A42EBD13A
:104D9C00254B1B6803F007033A689A420CD2224B4E
:104DAC003A68D2B21A70204B1B6803F007033A68BA
:104DBC009A4201D0012332E07B681B6803F00403A4
:104DCC00002B08D0194B9B6823F4E0527B68DB68FE
:104DDC00164913438B607B681B6803F00803002B98
:104DEC0009D0124B9B6823F460427B681B69DB0083
:104DFC000E4913438B6000F021F802460B4B9B6865
:104E0C001B0903F00F030A49CB5C22FA03F3094A8E
:104E1C001360094B1B681846FEF74CF90023184623
:104E2C001037BD4680BD00BF003C02400038024038
:104E3C00C0590008000000200C0000202DE9B04FE4
:104E4C0094B000AF00237B640023FB6400233B641D
:104E5C000023BB64794B9B6803F00C03082B0DD02B
:104E6C00082B00F2E180002B02D0042B03D0DBE0F6
:104E7C00734BBB64DBE0734BBB64D8E06F4B5B687C
:104E8C0003F03F037B646D4B5B6803F48003002BE2
:104E9C0063D06A4B5B689B090022BB63FA63BB6BF4
:104EAC00C3F308033B6300237B63D7E90C4522461D
:104EBC002B464FF000004FF00001590141EAD2613E
:104ECC00500102460B462146511A3961294663EBC3
:104EDC0001037B614FF000024FF00003D7E904ABF4
:104EEC0059468B01514643EA916351468A0151461A
:104EFC00B2EB0108594663EB01094FF000024FF089
:104F0C0000034FEAC90343EA58734FEAC8029046BC
:104F1C009946234618EB0303BB602B4649EB03036E
:104F2C00FB604FF000024FF00003D7E90245294621
:104F3C004B02214643EAD15321464A0210461946F8
:104F4C007B6C0022BB62FA62D7E90A23FBF738F9C3
:104F5C0002460B461346FB6458E0384B5B689B09D2
:104F6C00002218461146C0F308033B6200237B6203
:104F7C00D7E9088942464B464FF000004FF000013C
:104F8C00590141EAD261500102460B464146B2EB4F
:104F9C00010A494663EB010B4FF000024FF000038E
:104FAC004FEA8B1343EA9A634FEA8A12B2EB0A0474
:104FBC0063EB0B054FF000024FF00003EB0043EAEC
:104FCC005473E20014461D464346E3183B604B46BF
:104FDC0045EB03037B604FF000024FF00003D7E971
:104FEC00004529468B02214643EA915321468A0209
:104FFC00104619467B6C0022BB61FA61D7E9062387
:10500C00FBF7DEF802460B461346FB640B4B5B6862
:10501C001B0C03F0030301335B003B64FA6C3B6C29
:10502C00B2FBF3F3BB6402E0054BBB6400BFBB6C8B
:10503C0018465037BD46BDE8B08F00BF003802405F
:10504C000024F40000127A0080B582B000AF7860C2
:10505C007B68002B01D1012341E07B6893F83D3044
:10506C00DBB2002B06D17B68002283F83C207868E9
:10507C00FCF732F97B68022283F83D207B681A68C2
:10508C007B6804331946104600F07EFA7B680122D7
:10509C0083F846207B68012283F83E207B6801223E
:1050AC0083F83F207B68012283F840207B68012233
:1050BC0083F841207B68012283F842207B6801221F
:1050CC0083F843207B68012283F844207B6801220B
:1050DC0083F845207B68012283F83D200023184685
:1050EC000837BD4680BD000080B485B000AF786045
:1050FC007B6893F83D30DBB2012B01D001234EE0ED
:10510C007B68022283F83D207B681B68DA687B6829
:10511C001B6842F00102DA607B681B68234A9342E9
:10512C0022D07B681B68B3F1804F1DD07B681B6855
:10513C001F4A934218D07B681B681E4A934213D0B7
:10514C007B681B681C4A93420ED07B681B681B4A09
:10515C00934209D07B681B68194A934204D07B6840
:10516C001B68184A934211D17B681B689B6803F03B
:10517C000703FB60FB68062B10D07B681B681A6862
:10518C007B681B6842F001021A6007E07B681B68B1
:10519C001A687B681B6842F001021A6000231846EB
:1051AC001437BD465DF8047B704700BF000001401A
:1051BC000004004000080040000C004000040140C6
:1051CC00004001400018004080B584B000AF78600A
:1051DC007B681B68DB68FB607B681B681B69BB60BA
:1051EC00BB6803F00203002B20D0FB6803F0020322
:1051FC00002B1BD07B681B686FF002021A617B6866
:10520C0001221A777B681B689B6903F00303002B50
:10521C0003D0786800F099F905E0786800F08BF914
:10522C00786800F09CF97B6800221A77BB6803F061
:10523C000403002B20D0FB6803F00403002B1BD0CD
:10524C007B681B686FF004021A617B6802221A7774
:10525C007B681B689B6903F44073002B03D0786850
:10526C0000F073F905E0786800F065F9786800F0F3
:10527C0076F97B6800221A77BB6803F00803002BD1
:10528C0020D0FB6803F00803002B1BD07B681B6845
:10529C006FF008021A617B6804221A777B681B681E
:1052AC00DB6903F00303002B03D0786800F04DF9A1
:1052BC0005E0786800F03FF9786800F050F97B68F9
:1052CC0000221A77BB6803F01003002B20D0FB6878
:1052DC0003F01003002B1BD07B681B686FF01002CF
:1052EC001A617B6808221A777B681B68DB6903F4F8
:1052FC004073002B03D0786800F027F905E078683C
:10530C0000F019F9786800F02AF97B6800221A7706
:10531C00BB6803F00103002B0CD0FB6803F0010306
:10532C00002B07D07B681B686FF001021A6178684C
:10533C00FBF7F8FFBB6803F08003002B0CD0FB6875
:10534C0003F08003002B07D07B681B686FF0800292
:10535C001A61786800F0DEFABB6803F04003002B9A
:10536C000CD0FB6803F04003002B07D07B681B6854
:10537C006FF040021A61786800F0FBF8BB6803F02C
:10538C002003002B0CD0FB6803F02003002B07D06C
:10539C007B681B686FF020021A61786800F0B0FA25
:1053AC0000BF1037BD4680BD80B584B000AF7860BB
:1053BC0039600023FB737B6893F83C30012B01D1DF
:1053CC000223B4E07B68012283F83C207B68022234
:1053DC0083F83D207B681B689B68BB60BB6823F02F
:1053EC007703BB60BB6823F47F43BB607B681B689F
:1053FC00BA689A603B681B68B3F5005F3ED0B3F5A2
:10540C00005F00F28780B3F5805F00F08680B3F513
:10541C00805F7FD8702B1AD0702B7BD8602B50D02C
:10542C00602B77D8502B3CD0502B73D8402B58D0B6
:10543C00402B6FD8302B64D0302B6BD8202B60D006
:10544C00202B67D8002B5CD0102B5AD062E07B68E5
:10545C0018683B6899683B685A683B68DB6800F0E1
:10546C00B3F97B681B689B68BB60BB6843F0770330
:10547C00BB607B681B68BA689A604FE07B681868F1
:10548C003B6899683B685A683B68DB6800F09CF99C
:10549C007B681B689A687B681B6842F480429A6040
:1054AC003CE07B6818683B6859683B68DB681A46C7
:1054BC0000F010F97B681B685021184600F069F960
:1054CC002CE07B6818683B6859683B68DB681A46B7
:1054DC0000F02FF97B681B686021184600F059F921
:1054EC001CE07B6818683B6859683B68DB681A46A7
:1054FC0000F0F0F87B681B684021184600F049F971
:10550C000CE07B681A683B681B681946104600F073
:10551C0040F903E00123FB7300E000BF7B6801222C
:10552C0083F83D207B68002283F83C20FB7B1846E7
:10553C001037BD4680BD80B483B000AF786000BF2B
:10554C000C37BD465DF8047B704780B483B000AF68
:10555C00786000BF0C37BD465DF8047B704780B4A3
:10556C0083B000AF786000BF0C37BD465DF8047B9C
:10557C00704780B483B000AF786000BF0C37BD4675
:10558C005DF8047B7047000080B485B000AF786094
:10559C0039607B681B68FB607B68434A934213D07D
:1055AC007B68B3F1804F0FD07B68404A93420BD09D
:1055BC007B683F4A934207D07B683E4A934203D0B4
:1055CC007B683D4A934208D1FB6823F07003FB6073
:1055DC003B685B68FA681343FB607B68324A934212
:1055EC002BD07B68B3F1804F27D07B682F4A934236
:1055FC0023D07B682E4A93421FD07B682D4A93425E
:10560C001BD07B682C4A934217D07B682B4A934261
:10561C0013D07B682A4A93420FD07B68294A934265
:10562C000BD07B68284A934207D07B68274A934269
:10563C0003D07B68264A934208D1FB6823F440735D
:10564C00FB603B68DB68FA681343FB60FB6823F084
:10565C0080023B685B691343FB603B689A687B681C
:10566C00DA623B681A687B689A627B680E4A9342DE
:10567C0003D07B68104A934203D13B681A697B685C
:10568C001A637B681B6843F004027B681A607B68B2
:10569C0001225A617B68FA681A6000BF1437BD4654
:1056AC005DF8047B704700BF00000140000400401F
:1056BC0000080040000C0040000401400040014084
:1056CC00004401400048014000180040001C00400C
:1056DC000020004080B487B000AFF860B9607A60F9
:1056EC00FB681B6A7B61FB681B6A23F00102FB6889
:1056FC001A62FB689B693B613B6923F0F0033B61D9
:10570C007B681B013A6913433B617B6923F00A03F5
:10571C007B617A69BB6813437B61FB683A699A6168
:10572C00FB687A691A6200BF1C37BD465DF8047BC2
:10573C00704780B487B000AFF860B9607A60FB68DE
:10574C001B6A7B61FB681B6A23F01002FB681A6200
:10575C00FB689B693B613B6923F470433B617B684D
:10576C001B033A6913433B617B6923F0A0037B6104
:10577C00BB681B017A6913437B61FB683A699A61C8
:10578C00FB687A691A6200BF1C37BD465DF8047B62
:10579C00704780B485B000AF786039607B689B68D7
:1057AC00FB60FB6823F07003FB603A68FB681343F3
:1057BC0043F00703FB607B68FA689A6000BF1437FC
:1057CC00BD465DF8047B704780B487B000AFF860CD
:1057DC00B9607A603B60FB689B687B617B6923F4F2
:1057EC007F437B613B681A027B681A43BB68134397
:1057FC007A6913437B61FB687A699A6000BF1C3736
:10580C00BD465DF8047B704780B485B000AF78600E
:10581C0039607B6893F83C30012B01D102235AE0AC
:10582C007B68012283F83C207B68022283F83D20B0
:10583C007B681B685B68FB607B681B689B68BB6054
:10584C00FB6823F07003FB603B681B68FA6813432A
:10585C00FB607B681B68FA685A607B681B68214A8E
:10586C00934222D07B681B68B3F1804F1DD07B68BC
:10587C001B681D4A934218D07B681B681B4A9342D5
:10588C0013D07B681B681A4A93420ED07B681B6846
:10589C00184A934209D07B681B68174A934204D07C
:1058AC007B681B68154A93420CD1BB6823F08003BC
:1058BC00BB603B685B68BA681343BB607B681B6862
:1058CC00BA689A607B68012283F83D207B680022CD
:1058DC0083F83C20002318461437BD465DF8047B42
:1058EC00704700BF00000140000400400008004069
:1058FC00000C004000040140004001400018004032
:10590C0080B483B000AF786000BF0C37BD465DF843
:10591C00047B704780B483B000AF786000BF0C3755
:10592C00BD465DF8047B704702440346934200D1A8
:10593C00704703F8011BF9E770B50D4D0D4C641B56
:10594C00A4100026A64209D10B4D0C4C00F026F8F1
:10595C00641BA4100026A64205D170BD55F8043B6B
:10596C0098470136EEE755F8043B98470136F2E7C5
:10597C00F85D0008F85D0008F85D0008FC5D0008A3
:10598C000A44914200F1FF3300D1704710B511F871
:10599C00014B03F8014F9142F9D110BDF8B500BF8E
:1059AC00F8BC08BC9E467047F8B500BFF8BC08BCF4
:0459BC009E4670474C
:1059C00000000000000000000102030406070809AF
:1059D00000000000963007772C610EEEBA5109994D
:1059E00019C46D078FF46A7035A563E9A395649EA9
:1059F0003288DB0EA4B8DC791EE9D5E088D9D297CD
:105A00002B4CB609BD7CB17E072DB8E7911DBF9028
:105A10006410B71DF220B06A4871B9F3DE41BE844C
:105A20007DD4DA1AEBE4DD6D51B5D4F4C785D383A8
:105A300056986C13C0A86B647AF962FDECC9658A4C
:105A40004F5C0114D96C0663633D0FFAF50D088DA8
:105A5000C8206E3B5E10694CE44160D5727167A24C
:105A6000D1E4033C47D4044BFD850DD26BB50AA5A8
:105A7000FAA8B5356C98B242D6C9BBDB40F9BCACCC
:105A8000E36CD832755CDF45CF0DD6DC593DD1AB28
:105A9000AC30D9263A00DE518051D7C81661D0BF4C
:105AA000B5F4B42123C4B3569995BACF0FA5BDB8A8
:105AB0009EB802280888055FB2D90CC624E90BB14C
:105AC000877C6F2F114C6858AB1D61C13D2D66B6A8
:105AD0009041DC760671DB01BC20D2982A10D5EF0C
:105AE0008985B1711FB5B606A5E4BF9F33D4B8E868
:105AF000A2C9077834F9000F8EA8099618980EE10C
:105B0000BB0D6A7F2D3D6D08976C6491015C63E667
:105B1000F4516B6B62616C1CD83065854E0062F28B
:105B2000ED95066C7BA5011BC1F4088257C40FF5E7
:105B3000C6D9B06550E9B712EAB8BE8B7C88B9FC0B
:105B4000DF1DDD62492DDA15F37CD38C654CD4FB67
:105B50005861B24DCE51B53A7400BCA3E230BBD40B
:105B600041A5DF4AD795D83D6DC4D1A4FBF4D6D367
:105B70006AE96943FCD96E34468867ADD0B860DA0B
:105B8000732D0444E51D03335F4C0AAAC97C0DDD67
:105B90003C710550AA41022710100BBE86200CC98B
:105BA00025B56857B3856F2009D466B99FE461CEE7
:105BB0000EF9DE5E98C9D9292298D0B0B4A8D7C70B
:105BC000173DB359810DB42E3B5CBDB7AD6CBAC067
:105BD0002083B8EDB6B3BF9A0CE2B6039AD2B17483
:105BE0003947D5EAAF77D29D1526DB048316DC73DF
:105BF000120B63E3843B64943E6A6D0DA85A6A7A83
:105C00000BCF0EE49DFF099327AE000AB19E077DDE
:105C100044930FF0D2A3088768F2011EFEC2066902
:105C20005D5762F7CB67658071366C19E7066B6E5E
:105C3000761BD4FEE02BD3895A7ADA10CC4ADD6782
:105C40006FDFB9F9F9EFBE8E43BEB717D58EB060DE
:105C5000E8A3D6D67E93D1A1C4C2D83852F2DF4F82
:105C6000F167BBD16757BCA6DD06B53F4B36B248DE
:105C7000DA2B0DD84C1B0AAFF64A0336607A044182
:105C8000C3EF60DF55DF67A8EF8E6E3179BE6946DE
:105C90008CB361CB1A8366BCA0D26F2536E2685202
:105CA00095770CCC03470BBBB91602222F2605555E
:105CB000BE3BBAC5280BBDB2925AB42B046AB35C82
:105CC000A7FFD7C231CFD0B58B9ED92C1DAEDE5BDE
:105CD000B0C2649B26F263EC9CA36A750A936D02C2
:105CE000A906099C3F360EEB85670772135700051E
:105CF000824ABF95147AB8E2AE2BB17B381BB60C42
:105D00009B8ED2920DBED5E5B7EFDC7C21DFDB0B9D
:105D1000D4D2D38642E2D4F1F8B3DD686E83DA1FC1
:105D2000CD16BE815B26B9F6E177B06F7747B7181D
:105D3000E65A0888706A0FFFCA3B06665C0B0111C1
:105D4000FF9E658F69AE62F8D3FF6B6145CF6C161D
:105D500078E20AA0EED20DD75483044EC2B30339C1
:105D6000612667A7F71660D04D476949DB776E3E1D
:105D70004A6AD1AEDC5AD6D9660BDF40F03BD83741
:105D800053AEBCA9C59EBBDE7FCFB247E9FFB5309D
:105D90001CF2BDBD8AC2BACA3093B353A6A3B424C1
:105DA0000536D0BA9306D7CD2957DE54BF67D9231D
:105DB0002E7A66B3B84A61C4021B685D942B6F2AC1
:105DC00037BE0BB4A18E0CC31BDF055A8DEF022D1D
:105DD00046004600960046009600010000000000C4
:105DE0000000000001070000090700005500010045
:085DF0000CA4FF7F010000007C
:045DF800B1010008ED
:045DFC008D0100080D
:105E00000024F400FFFFFFFFF1020000100000007B
:045E1000010000008D
:0400000508001409D2
:00000001FF
